:020000000528D1
:10000800B5288B138312031383120313850186010A
:100018008316FF30831603138500FF308600831292
:100028008B138730831681008312C3308312031326
:10003800B600B7018100A0308B00B801FF30BB01CA
:10004800BC01BD00BE004B2883120313BA00031085
:10005800380D3B3E8400831339088000840A3A082F
:100068008000B80A3808013A0319B8010310380D9E
:1000780083133B3E84000008840A000403193528D2
:10008800801B352800088A00840300088200831634
:100098000313850186018312031385018601073046
:1000A8009F000311031959285A28AF2883120313F4
:1000B8008501A8010310A81B632805302802031C2A
:1000C80066288D2883120313A401A501A601A701A0
:1000D800031427082604031D792813302502031C5E
:1000E8007928031D792888302402031C7C28872856
:1000F80083120313A901A40A0319A50A0319A60A5E
:100108000319A70A6C280130831203138506A80A6D
:100118005E2883120313A401A501A601A7010314F5
:1001280027082604031DA0284E302502031CA028FA
:10013800031DA02820302402031CA328AE28831204
:100148000313A901A40A0319A50A0319A60A031986
:10015800A70A932855288312031323088A00220824
:100168008200FF00030E8312031383120313B000EF
:10017800B00E0A08B1000408B2000B1DD4283608D6
:1001880081005030B707B4300318013EFF3A013EF2
:10019800B6000B11FF30BE1BD428BD07031CBE07D9
:1001A8007C08B3007D08B4007E08B5003508FE0061
:1001B8003408FD003308FC003208840031088A0046
:0A01C80030088300FF0E7F0E0900CF
:02400E00103F61
:00000001FF
